:1000000000308A0071290000FF00030E8301A10067
:100010007F08A0000A08A8008A01A00E0408A20018
:100020007708A3007808A4007908A5007A08A6003C
:100030007B08A700831383128C308400801D222844
:100040008C193528220884002308F7002408F800BA
:100050002508F9002608FA002708FB0028088A006E
:10006000210E8300FF0E7F0E09008A114C280A1012
:100070008A100A118207023406340E341E343E34CC
:100080007E34FE34FF340A108A100A11820741348C
:1000900068346F346A340034680893008C118A1114
:1000A00022286D3084000008031963280130F8000D
:1000B000F701F70B5928F80B58283A30F700F70BDF
:1000C0005F28800B56280034831605178312051FFE
:1000D0006B2805136C2805178316051383128A11E4
:1000E000012A690884006D088000840A8001E90AF9
:1000F0008A110D2ABC01391C7F2839108028391437
:100100000034391CAB2883168612831286124530C0
:10011000F700F70B8928000000008316861283126F
:1001200086164530F700F70B932800000000831671
:100130008612831286124530F700F70B9D280000C7
:10014000000083168612831286161830F700F70B0C
:10015000A7280000BD2883168612831286128230DB
:10016000F700F70BB12883168612831286166C30BF
:10017000F700F70BB928000000000034EF016F080A
:10018000073C031C06296E080139F000BE0803195C
:10019000CB280030CC280130F100BD080319D2284B
:1001A0000030D32801307105003A0319E6287008A1
:1001B000F1000310BB0CBA0C030801397106013CB5
:1001C000031DE6288430BB060830BA06F008031D7C
:1001D000EB287A200129BD080319BC0ABD080319C0
:1001E000F3280030F4280130F1003C08053C0319E5
:1001F000FB280030FC2801307105031901298120FA
:100200007A2081200310EE0CEF0ABF280034391049
:10021000FF30BB00BA00BC010130BD00BE01BF0110
:100220003F08093C031C19297E30EE00BE20BF0A9E
:100230001029BD01BF013F080F3C031C28292930AC
:100240003F0784000008ED00EE00BE20BF0A1B2916
:10025000BF016C0884000008031937296C0884006A
:100260000008ED00EE00BE20EC0ABF0A292901308B
:10027000BE00FF30BA06BB063A08EE00BE203B08BF
:10028000EE00BE20BE010130BD007E30EE00BE207B
:100290008A11112AED016D08F93C031C68296C18BC
:1002A00053290513542905178316051301308312AA
:1002B000EC066C185D2985135E2985178316851356
:1002C0001F30F700F70B622900008312ED0A4B295B
:1002D000831605138312051783168513831285175A
:1002E000003484011F30830583161F129F121B08E0
:1002F00080399B0007309C0082308312A90098301F
:10030000AA00AB004030AC00AD00AE006030AF00E2
:100310008630B000B430B1006030B200A430B30019
:10032000B400B5006130B6000330B700F030B8005B
:10033000E90183161F129F121B088039D0389B00D9
:100340001F1383121F179F1783169F1383121F14E7
:10035000941283160611861406120030831294003C
:10036000831694000108C039073881008312900178
:10037000073083169C0005080230F700F70BBE29F2
:10038000000000001C0883120D1383169D018611C6
:1003900083128611831606118312061183168610A6
:1003A000831286108316851383128517831605130F
:1003B000831205172030F8001F08C73978049F0002
:1003C000950183168611831286110C309700003038
:1003D000F8000438920064308316920062308F0077
:1003E000023083129500EA0183168610831286106C
:1003F0006430ED0051206A08EA0A043C031D112A0A
:100400006428EA014030E900EC016C084320003820
:1004100003190E2AEC0AED007128052A4030EC0081
:10042000072983168610831286140130ED005120AF
:100430001F151F19192A1E08503C031CF429831686
:100440008610831286104A216430EB00EA016A08A4
:10045000073C031C4D2A95010030F8000438920037
:100460006B08831692001330831295006430ED0000
:10047000512083168610831286140130ED0051201E
:100480001F151F19412A1E086A3C0318EB03831627
:10049000861083128610EA0A272A3A30EC00FA30D6
:1004A000ED005120EC0B4F2A831694012230831269
:1004B00094000230E80068089300C0308B04831673
:1004C0008C158312EA016A08073C031C702A6A082B
:1004D0003720F800E8003C30ED005120EA0A632A9A
:1004E000831694018312940183168C1106118312D2
:1004F00006150430EC00FA30ED005120EC0B7B2A9D
:10050000831606118312061195014A210830EC006A
:10051000FA30ED005120EC0B882A4A21831606118F
:100520008312061583168513831285178316051308
:10053000831205130230EC009630ED005120EC0BD5
:100540009C2A831685138312851383160513831241
:1005500005170230EC009630ED005120EC0BAB2A71
:10056000922A1430EC00FA30ED005120EC0BB32A43
:060570008A01002863006F
:04400E003827FC3F14
:00000001FF
